:107000000C945D380C9495380C947A380C947A383A
:107010000C947A380C947A380C947A380C947A3828
:107020000C947A380C947A380C947A380C947A3818
:107030000C947A380C947A380C947A380C947A3808
:107040000C947A380C947A380C947A380C947A38F8
:107050000C947A380C947A380C947A380C947A38E8
:107060000C947A380C947A38040309041C037700D2
:10707000770077002E0066006900730063006800E7
:107080006C002E00640065000E03550053004200A2
:1070900061007300700012011001FF000008C016AB
:1070A000DC05020101020001090212000101008059
:1070B000FA09040000000000000011241FBECFEFF9
:1070C000D8E0DEBFCDBF11E0A0E0B1E0E4E1F8E739
:1070D00002C005900D92A630B107D9F711E0A6E0E5
:1070E000B1E001C01D92AC33B107E1F70E94EB396A
:1070F0000C94083C0C940038A82FB92F80E090E045
:1071000041E050EA609530E009C02D9182279795C3
:10711000879510F084279527305EC8F36F5FA8F33A
:107120000895EADF8D939D930895CF93CFB7CF93C2
:10713000C3954F9BE9F74F9B0BC04F9B09C04F9BDB
:1071400007C04F9B05C04F9B03C04F9B01C0C0C0F1
:10715000C0911F01DF93DD27CA5DDE4F2F932FEF14
:107160004F9B03C02F91DF91E6CF0F931F934F9357
:107170006F9309B107FB20F93F933BE05F931EC07B
:107180004E7F012F19B11478E1F0216000001DC07D
:10719000102F4D7F2260000009B1047891F01DC0CE
:1071A0004B7F2460012F000019B1147851F01EC0EC
:1071B00019B1147831F0477F28601BC019B11478D9
:1071C00009F462C04FEF297FD9F2012707FB21F9AB
:1071D00009B10478B1F3237FD9F2102717FB22F904
:1071E00000C019B1147869F3277ED1F2012707FB9B
:1071F00023F92F7CE9F209B1047819F3102717FB62
:1072000024F92F7929F100C019B11478E9F1012787
:1072100007FB25F92F7311F100C009B10478A1F122
:10722000102717FB26F92230F8F000C019B11478A6
:1072300059F1012707FB27F92430E0F0422700002D
:1072400009B14993102717FB20F93150C8F0B6CF88
:107250004F7E09B10478C1F02061D3CF206219B10B
:10726000147891F04F7DD6CF4F7B09B1047861F04F
:107270002064D9CF4F7719B1147831F02068DCCF72
:1072800011E01CBB002717C03B503195C31BD040F9
:1072900011E01CBB0881033CF9F00B34E9F02091AC
:1072A0001D011981110F1213EDCF093651F10D3265
:1072B00011F0013E39F7009324015F913F916F91E6
:1072C0004F911F910F912F91DF91CCB3C0FD30CF23
:1072D000CF91CFBFCF91189520912401222369F33C
:1072E00010912201112331F5343032F13093220113
:1072F00020931E0110911F013BE0311B30931F01B1
:107300001BC0009122010130ACF40AE5309100016C
:1073100034FD13C000930001C2E1D1E012C0052783
:107320001127000019C0052711271FC005271127A5
:10733000000024C04AE502C032ED432FC4E1D0E092
:1073400032E01AB114685F9A0BB11AB954E820E818
:1073500066E020FF052727950BB917951C3FF8F627
:107360006A95B9F720FF0527279500000BB91795F7
:107370001C3FC8F620FF05272795179566E01C3FA0
:107380000BB9A0F629913A9521F70B7710912301BB
:10739000110F0BB9C651D04011F010931D0111E02F
:1073A0001CBB00681AB11B77402F4B7753E05A95EE
:1073B000F1F700C00BB91AB94BB97FCF1BB8F894DD
:1073C0001DBA1092690081E085BF15BEE0911001E1
:1073D000F091110109952F923F924F925F926F9217
:1073E0007F928F929F92AF92BF92CF92DF92EF9255
:1073F000FF920F931F93CF93DF9388E10FB6F8941A
:1074000080936000109260000FBE5F9A04B601FE88
:10741000E7C114BE81E085BF82E085BF4F99E0C11E
:1074200080916900836080936900E89A4F9BFECF4A
:10743000579878946CE0262E312C03E058E8C52E3E
:1074400050E7D52E4CE6A42E40E7B42E38E6832E26
:1074500030E7932E28EA622E20E7722E96E9492E15
:1074600090E7592E87E0E82E81E0F82E90912201D6
:10747000935097FD29C180911F01E101C81BD109DB
:10748000CA5DDE4F80911E018D3209F0C1C0983077
:1074900009F018C123EC209312018AE580930001C2
:1074A00010920B013881832F80762981882309F47B
:1074B00044C0F0922101E09220012330D9F49B8155
:1074C0008C812A81203339F48370E82FF0E0EE5F5D
:1074D000FE4F80810BC0203A19F40E94F23B06C097
:1074E000203C19F46D810E94FA3B80E080930A01F0
:1074F00094E07EC0253011F491E07AC0822F845050
:107500008630A0F48A819B8190930D0180930C01B9
:10751000293009F46CC09E8190930E018D81827098
:1075200080930F0137FD68C02FEF67C0223009F04C
:107530005EC0E1E0E09306015AC08A8110921B010F
:10754000222331F410921C012BE131E092E04AC079
:10755000253019F48093230142C0263081F58B81B8
:10756000813029F4509221014092200106C08230DE
:1075700031F4709221016092200192E11CC08330AD
:10758000C9F48A81882331F49092210180922001EC
:1075900094E011C0813031F4B0922101A092200119
:1075A0009CE109C0823031F4D0922101C0922001C7
:1075B0009EE001C090E0F0E4F0930B0119C0283088
:1075C00019F425E231E009C0293019F4809325012E
:1075D00006C02A3021F42BE131E091E003C02BE119
:1075E00031E090E0309321012093200101C090E030
:1075F0008F81882331F008C0292F80E880930B0108
:1076000004C02E81291708F0292F209301015AC0A8
:1076100080910B0187FF56C080910E01592F891769
:1076200008F4582F851B80930E0160E0882309F42D
:1076300061E070910F01E0910C01F0910D0140E0CB
:1076400036C0CF018F779070892B41F4F894009366
:107650005700E895789407B600FCFDCF4E5FF8948C
:107660008991999121E00C0120935700E89511240C
:1076700078949F012E5F3F4FC9018F779070892BBF
:1076800031F0662399F0451788F0772379F0F89464
:1076900085E080935700E895789407B600FCFDCF0D
:1076A000F894E1E1E0935700E8957894F9014517E3
:1076B00008F4C7CFF0930D01E0930C01662311F09D
:1076C00010920101109222018091000184FF79C083
:1076D000809101018F3F09F474C0182F893008F0A0
:1076E00018E0811B809301018091120198E889279D
:1076F00080931201112309F451C080910B0187FF7F
:107700001EC080910E01811708F4182F811B8093F1
:107710000E01A0910C01B0910D01AD01C3E1D1E0CA
:10772000212F30E0B9016C0F7D1F05C0FA01849153
:1077300089934F5F5F4FC617D707C1F727C02091C6
:1077400020013091210186FF0DC0A3E1B1E080E06E
:1077500090E0F901E80FF91FE491ED9301961817F5
:10776000C1F708C0D901912FE3E1F1E08D91819338
:107770009150E1F71150812F90E01F5F0196820F29
:10778000931F909321018093200108C02A0F3B1F73
:1077900030930D0120930C01193068F483E191E0DE
:1077A000612F0E949138612F6C5F6C3041F08FEF38
:1077B0008093010104C08FEF809301016EE160931B
:1077C000000194E189B1847831F49150D9F7109295
:1077D000230110921D0180910601882309F446CEF1
:1077E0000E94DE39F999FECF92BD81BDF89A9927A2
:1077F00080B50895262FF999FECF1FBA92BD81BD9D
:1078000020BD0FB6F894FA9AF99A0FBE0196089522
:04781000F894FFCF1A
:067814005AFF1E950F0053
:040000030000700089
:00000001FF
